:020000040000FA
:04000000AEEF0AF065
:0400080089EF06F086
:06002A00D9CFE5FFE1CF94
:10003000D9FF00C0E5FF01C0E5FF02C0E5FF03C036
:10004000E5FF04C0E5FF05C0E5FF06C0E5FF07C00A
:10005000E5FF08C0E5FF09C0E5FF0AC0E5FF020EA5
:10006000DBCF00F0030EDBCF01F0040EDBCF02F09C
:10007000050EDBCF03F0060EDBCF04F0070EDBCF5F
:1000800005F000C006F001C007F002C008F0035000
:1000900003E003500508036E270EE56E100EE56EB3
:1000A0000550E56E0450E56E44EC05F0096EF3CFA3
:1000B0000AF0040EE126300E092609C0E5FF06C04D
:1000C000E9FF07C0F3FF0850BAEC0AF0062AD8B0DF
:1000D000072AD8B0082A030603500EE12E0EE56E5B
:1000E00006C0E9FF07C0F3FF0850BAEC0AF0062A81
:1000F000D8B0072AD8B0082A270EE56E100EE56E94
:100100000550E56E0450E56EE8EC04F0046EF3CFA4
:1001100005F0040EE126030EE56EE80EE56E0550CF
:10012000E56E0450E56E44EC05F0096EF3CF0AF07D
:10013000040EE126300E092609C0E5FF06C0E9FFDE
:1001400007C0F3FF0850BAEC0AF0062AD8B0072A15
:10015000D8B0082A030603500EE12E0EE56E06C045
:10016000E9FF07C0F3FF0850BAEC0AF0062AD8B03E
:10017000072AD8B0082A030EE56EE80EE56E055092
:10018000E56E0450E56EE8EC04F0046EF3CF05F084
:10019000040EE126000EE56E640EE56E0550E56E78
:1001A0000450E56E44EC05F0096EF3CF0AF0040E3E
:1001B000E126300E092609C0E5FF06C0E9FF07C0A9
:1001C000F3FF0850BAEC0AF0062AD8B0072AD8B0D4
:1001D000082A030603500EE12E0EE56E06C0E9FF65
:1001E00007C0F3FF0850BAEC0AF0062AD8B0072A75
:1001F000D8B0082A000EE56E640EE56E0550E56E77
:100200000450E56EE8EC04F0046EF3CF05F0040E44
:10021000E126000EE56E0A0EE56E0550E56E04500F
:10022000E56E44EC05F0096EF3CF0AF0040EE1260A
:10023000300E092609C0E5FF06C0E9FF07C0F3FF3D
:100240000850BAEC0AF0062AD8B0072AD8B0082A13
:10025000030603500EE12E0EE56E06C0E9FF07C04F
:10026000F3FF0850BAEC0AF0062AD8B0072AD8B033
:10027000082A000EE56E0A0EE56E0550E56E045084
:10028000E56EE8EC04F0046EF3CF05F0040EE12611
:10029000300E042604C0E5FF06C0E9FF07C0F3FFE7
:1002A0000850BAEC0AF0062AD8B0072AD8B0082AB3
:1002B000032E09D02E0EE56E06C0E9FF07C0F3FF3E
:1002C0000850BAEC0AF00050040F036E000E012033
:1002D000046E000E0220056E0250800FF36E055072
:1002E000800FF35C05E10450015C02E10350005C07
:1002F00019E200C0E9FF01C0F3FF025056EC0AF01A
:10030000066E300A0FE1200EE56E00C0E9FF01C065
:10031000F3FF0250BAEC0AF0002AD8B0012AD8B094
:10032000022ADAD7E4CF0AF0E4CF09F0E4CF08F0EC
:10033000E4CF07F0E4CF06F0E4CF05F0E4CF04F01B
:10034000E4CF03F0E4CF02F0E4CF01F0E4CF00F01B
:10035000E4CFD9FF1200D9CFE5FFE1CFD9FF00C02C
:10036000E5FF01C0E5FF02C0E5FF03C0E5FF04C0F3
:10037000E5FF05C0E5FF06C0E5FF07C0E5FF020E8B
:10038000DBCF00F0030EDBCF01F0040EDBCF02F079
:10039000050EDBCF03F0640EE56E03C0E5FFA9ECAC
:1003A00008F0046EE450E450300E042604C0E5FF6B
:1003B00000C0E9FF01C0F3FF0250BAEC0AF00050A0
:1003C000010F046E000E0120056E000E0220066E65
:1003D000640EE56E03C0E5FFFFEC07F0036EE4502A
:1003E000E4500A0EE56E03C0E5FFA9EC08F0076EC5
:1003F000E450E450300E072607C0E5FF04C0E9FFD3
:1004000005C0F3FF0650BAEC0AF0042AD8B0052A5A
:10041000D8B0062A0A0EE56E03C0E5FFFFEC07F030
:10042000036EE450E450300E032603C0E5FF04C021
:10043000E9FF05C0F3FF0650BAEC0AF00050020FC6
:10044000036E000E0120046E000E0220056E0250A5
:10045000800FF36E0550800FF35C05E10450015CE2
:1004600002E10350005C19E200C0E9FF01C0F3FFA4
:10047000025056EC0AF0066E300A0FE1200EE56ECF
:1004800000C0E9FF01C0F3FF0250BAEC0AF0002AF5
:10049000D8B0012AD8B0022ADAD7E4CF07F0E4CFE7
:1004A00006F0E4CF05F0E4CF04F0E4CF03F0E4CFAE
:1004B00002F0E4CF01F0E4CF00F0E4CFD9FF120066
:1004C000D9CFE5FFE1CFD9FF00C0E5FF01C0E5FFCF
:1004D00002C0E5FF03C0E5FF04C0E5FF05C0E5FF7E
:1004E00006C0E5FF07C0E5FF08C0E5FF020EDBCF51
:1004F00000F0030EDBCF01F0040EDBCF02F0050E9F
:10050000DBCF03F0060EDBCF04F0070EDBCF05F0E8
:10051000080EDBCF06F0090EDBCF07F0ACEC09F0DC
:1005200003A003D0020EC86E02D0090EC86EF5EC0F
:100530000AF00050E56EA2EC0AF0E12A03A208D00E
:100540000250036E086A0350E56EA2EC0AF0E12A3D
:100550000150E56EA2EC0AF0E12AEFEC0AF000800F
:100560000050E56EA2EC0AF0E12A04C000F005C0DC
:1005700001F006C002F007C003F0020E035C16E3B0
:10058000010EE56EFBEC09F0046EE12A04C0E5FF04
:1005900000C0E9FF01C0F3FF0250BAEC0AF0002AE4
:1005A000D8B0012AD8B0022A0306E7D703500FE0DB
:1005B000000EE56EFBEC09F0036EE12A03C0E5FFD7
:1005C00000C0E9FF01C0F3FF0250BAEC0AF0E9EC09
:1005D0000AF0E86AE4CF08F0E4CF07F0E4CF06F0D1
:1005E000E4CF05F0E4CF04F0E4CF03F0E4CF02F071
:1005F000E4CF01F0E4CF00F0E4CFD9FF1200D9CF6F
:10060000E5FFE1CFD9FF00C0E5FF01C0E5FF02C073
:10061000E5FF03C0E5FF04C0E5FF05C0E5FF06C038
:10062000E5FF07C0E5FF08C0E5FF09C0E5FF0AC018
:10063000E5FF0BC0E5FF0CC0E5FF0DC0E5FF020EB6
:10064000DBCF00F0030EDBCF01F0040EDBCF02F0B6
:10065000050EDBCF03F0060EDBCF04F0070EDBCF79
:1006600005F0080EDBCF06F0090EDBCF07F0086AB5
:10067000096A0A6A0B6A200E0C6E0344010B0D6EA8
:10068000010E0D16005000260136023603360850C2
:10069000082609360A360B360D50D8A408800750B4
:1006A0000B5C08E106500A5C05E10550095C02E1BB
:1006B0000450085C09E30450085E0550095A0650CE
:1006C0000A5A07500B5A00800C2ED7D703C0E9FFF7
:1006D00002C0F4FF01C0F3FF0050E4CF0DF0E4CFFF
:1006E0000CF0E4CF0BF0E4CF0AF0E4CF09F0E4CF54
:1006F00008F0E4CF07F0E4CF06F0E4CF05F0E4CF54
:1007000004F0E4CF03F0E4CF02F0E4CF01F0E4CF53
:1007100000F0E4CFD9FF1200D9CFE5FFE1CFD9FF38
:1007200000C0E5FF01C0E5FF02C0E5FF03C0E5FF33
:1007300004C0E5FF05C0E5FF06C0E5FF07C0E5FF13
:10074000020EDBCF00F0030EDBCF01F0040EDBCF97
:1007500002F0050EDBCF03F0060EDBCF04F0070E30
:10076000DBCF05F0080EDBCF06F0090EDBCF07F07C
:10077000ACEC09F003A003D0020EC86E02D0090E43
:10078000C86EF5EC0AF00050E56EA2EC0AF0E12A22
:1007900003A208D00250006E036A0050E56EA2EC7E
:1007A0000AF0E12A0150E56EA2EC0AF0E12A04C049
:1007B00000F005C001F006C002F007C003F003C05E
:1007C00004F00306045013E000C0E9FF01C0F3FF8A
:1007D000025056EC0AF0046E002AD8B0012AD8B0B4
:1007E000022A0450E56EA2EC0AF0E12AE8D7E9EC0F
:1007F0000AF0E86AE4CF07F0E4CF06F0E4CF05F0B2
:10080000E4CF04F0E4CF03F0E4CF02F0E4CF01F052
:10081000E4CF00F0E4CFD9FF1200D9CFE5FFE1CF5C
:10082000D9FF00C0E5FF01C0E5FF02C0E5FF03C03E
:10083000E5FF04C0E5FF020EDBCF00F0030EDBCFC7
:1008400001F0040EDBCF02F0050EDBCF03F0060E45
:10085000DBCF04F0ACEC09F0090EC86EF5EC0AF041
:10086000C60EE56EA2EC0AF0E12A000EE56EA2ECDF
:100870000AF0E12AFE0EE56EA2EC0AF0E12A015030
:10088000400DF3CF01F0800E0126015000260050EC
:10089000E56EA2EC0AF0E12A02C000F003C001F00C
:1008A00004C002F000C0E9FF01C0F3FF025056ECA3
:1008B0000AF0036E03500BE0002AD8B0012AD8B02A
:1008C000022A0350E56EA2EC0AF0E12AEBD7FF0EF4
:1008D000E56EA2EC0AF0E12AE9EC0AF0000EE56E02
:1008E0000A0EE56E7EEC09F0020EE126E4CF04F07C
:1008F000E4CF03F0E4CF02F0E4CF01F0E4CF00F066
:10090000E4CFD9FF1200D9CFE5FFE1CFD9FF00C076
:10091000E5FF01C0E5FF02C0E5FF03C0E5FF04C03D
:10092000E5FF05C0E5FF06C0E5FF07C0E5FF08C01D
:10093000E5FF09C0E5FF0AC0E5FF0BC0E5FF020EB9
:10094000DBCF00F00050E56E8BEC07F0016EF3CFCB
:1009500002F0E12A036A046A002A002A0050E56EC8
:100960008BEC07F0006EF3CF05F0E12A066A076A08
:1009700005500B6E00500A6E086A096A0850011291
:10098000095002120A5003120B50041204C0E9FF6E
:1009900003C0F4FF02C0F3FF0150E4CF0BF0E4CF3B
:1009A0000AF0E4CF09F0E4CF08F0E4CF07F0E4CF99
:1009B00006F0E4CF05F0E4CF04F0E4CF03F0E4CF99
:1009C00002F0E4CF01F0E4CF00F0E4CFD9FF120051
:1009D000D9CFE5FFE1CFD9FF00C0E5FF01C0E5FFBA
:1009E00002C0E5FF03C0E5FF04C0E5FF05C0E5FF69
:1009F00006C0E5FF020EDBCF00F0030EDBCF01F0F7
:100A0000040EDBCF02F0050EDBCF03F0046A056AAB
:100A10000344010B066E06B011D0025002260336C5
:100A20000350015C02E10250005C04E2D890033202
:100A3000023204D0052A05C004F0EAD70350015C55
:100A400002E10250005C04E30250005E0350015AD0
:100A5000D8900332023204C005F004060550EEE1DE
:100A600001C0F3FF0050E4CF06F0E4CF05F0E4CF7F
:100A700004F0E4CF03F0E4CF02F0E4CF01F0E4CFE0
:100A800000F0E4CFD9FF1200D9CFE5FFE1CFD9FFC5
:100A900000C0E5FF01C0E5FF02C0E5FF03C0E5FFC0
:100AA00004C0E5FF05C0E5FF06C0E5FF07C0E5FFA0
:100AB000020EDBCF00F0030EDBCF01F0040EDBCF24
:100AC00002F0050EDBCF03F0046A056A100E066E15
:100AD0000144010B076E010E071600500026013677
:100AE0000450042605360750D8A404800350055C42
:100AF00002E10250045C05E30250045E0350055A13
:100B00000080062EE5D701C0F3FF0050E4CF07F0C8
:100B1000E4CF06F0E4CF05F0E4CF04F0E4CF03F037
:100B2000E4CF02F0E4CF01F0E4CF00F0E4CFD9FF4E
:100B30001200D9CFE5FFE1CFD9FF00C0E5FF01C02A
:100B4000E5FF02C0E5FF020EDBCF00F000380F0B1F
:100B5000016E300E01263A0E015C02E3070E0126FB
:100B600001500001836F0F0E0014016E300E01263C
:100B70003A0E015C02E3070E012601500001846F6A
:100B80008569000E016E830E006E800E026E030EEC
:100B9000E56E0250E56E0150E56E0050E56E000E08
:100BA000E56E000EE56E000EE56EC60EE56E8CEC91
:100BB00003F0080EE126000EE56E0A0EE56E7EECEF
:100BC00009F0020EE126E4CF02F0E4CF01F0E4CF19
:100BD00000F0E4CFD9FF1200D9CFE5FFE1CFD9FF74
:100BE00000C0E5FF01C0E5FF02C0E5FF03C0E5FF6F
:100BF00004C0E5FF05C0E5FF06C0E5FF020EDBCF40
:100C000000F0030EDBCF01F0040EDBCF02F0050E87
:100C1000DBCF03F0060EDBCF04F00150056E02506F
:100C2000066EE56E0550E56E0050E56E50EC07F07F
:100C3000030EE126002A002A0350016E0450026EC2
:100C4000036A046A0250E56E0150E56E0050E56EDD
:100C500050EC07F0030EE126E4CF06F0E4CF05F0F8
:100C6000E4CF04F0E4CF03F0E4CF02F0E4CF01F0EE
:100C7000E4CF00F0E4CFD9FF1200B80EF66E150EE7
:100C8000F76E000EF86E0900F550056E0900F5507C
:100C9000066E055002E106503BE00900F550006E7B
:100CA0000900F550016E0900F550026E09000900B7
:100CB000F550E96E0900F550EA6E090009000900D7
:100CC000F550036E0900F550046E09000900F6CFD7
:100CD00007F0F7CF08F0F8CF09F000C0F6FF01C029
:100CE000F7FF02C0F8FF035002E1045007E00900DB
:100CF000F550EE6E0306F8E20406F9D707C0F6FFDA
:100D000008C0F7FF09C0F8FF0506C4E20606C5D70C
:100D10001200E8CFE5FFD8CFE5FFE0CFE5FFF3CF46
:100D2000E5FFF4CFE5FFE9CFE5FFEACFE5FFFACF36
:100D3000E5FFFBCFE5FF00C0E5FFA1A21DD0FBEC66
:100D40000AF08AC000F000018A2B00500A0A13E161
:100D5000006A81BE002A0050D880E866D890006AF8
:100D600000360050010BE840F46E81507F0BF41008
:100D7000816E00018A6BA192E4CF00F0E4CFFBFF0B
:100D8000E4CFFAFFE4CFEAFFE4CFE9FFE4CFF4FFDA
:100D9000E4CFF3FFE4CFE0FFE4CFD8FFE4CFE8FFF8
:100DA0001000D9CFE5FFE1CFD9FF00C0E5FF01C0BA
:100DB000E5FF02C0E5FF03C0E5FF04C0E5FF05C095
:100DC000E5FF020EDBCF00F0030EDBCF01F0040ED7
:100DD000DBCF02F0050EDBCF03F0046A0350045CA6
:100DE00014E200C0E9FF01C0F3FF025056EC0AF024
:100DF000056E002AD8B0012AD8B0022A0550E56E47
:100E000044EC0AF0E12A042AE9D7E4CF05F0E4CF64
:100E100004F0E4CF03F0E4CF02F0E4CF01F0E4CF3C
:100E200000F0E4CFD9FF1200D9CFE5FFE1CFD9FF21
:100E300000C0E5FF01C0E5FF02C0E5FF020EDBCF09
:100E400000F000500001866F8769000E016E860E6B
:100E5000006E800E026E020EE56E0250E56E0150CD
:100E6000E56E0050E56E000EE56E000EE56E000EBC
:100E7000E56EC60EE56E8CEC03F0080EE126000E62
:100E8000E56E0A0EE56E7EEC09F0020EE126E4CF77
:100E900002F0E4CF01F0E4CF00F0E4CFD9FF12007C
:100EA000D9CFE5FFE1CFD9FF00C0E5FF01C0E5FFE5
:100EB00002C0E5FF020EDBCF00F0030EDBCF01F036
:100EC000040EDBCF02F0A69EA69CA684F29E00C074
:100ED000A9FF0150A86E550EA76EAA0EA76EA68296
:100EE000A6B2FED70028A96E0250016E026A015018
:100EF000A86E550EA76EAA0EA76EA682A6B2FED742
:100F0000A694F28EE4CF02F0E4CF01F0E4CF00F03B
:100F1000E4CFD9FF1200D9CFE5FFE1CFD9FF00C060
:100F2000E5FF01C0E5FF02C0E5FF03C0E5FF04C027
:100F3000E5FF05C0E5FF020EDBCF00F0A69CA69EF4
:100F400000C0A9FFA680A8CF01F0026A0028A96E00
:100F5000A680A8CF00F0036A0050056E046A045012
:100F600001120550021202C0F3FF0150E4CF05F058
:100F7000E4CF04F0E4CF03F0E4CF02F0E4CF01F0DB
:100F8000E4CF00F0E4CFD9FF1200D9CFE5FFE1CFE5
:100F9000D9FF00C0E5FF01C0E5FF02C0E5FF03C0C7
:100FA000E5FF020EDBCF00F0030EDBCF01F0040EF5
:100FB000DBCF02F000C0E9FF01C0F3FF025056ECA6
:100FC0000AF0036E035010E0ACA2FED700C0E9FFA8
:100FD00001C0F3FF025056EC0AF0AD6E002AD8B003
:100FE000012AD8B0022AE6D7E4CF03F0E4CF02F01A
:100FF000E4CF01F0E4CF00F0E4CFD9FF1200D9CF65
:10100000E5FFE1CFD9FF00C0E5FF01C0E5FF02C069
:10101000E5FF03C0E5FF020EDBCF00F0030EDBCFE0
:1010200001F0026A036A01BE0CD0D890013601506B
:10103000005C03E2D890013204D0032A03C002F01E
:10104000F2D70150005C02E30150005ED8900132FB
:1010500002C003F002060350F4E10050E4CF03F0B5
:10106000E4CF02F0E4CF01F0E4CF00F0E4CFD9FF09
:10107000120000C0E5FF01C0E5FF02C0E5FF03C0AC
:10108000E5FFE0EC08F0006EF3CF01F0F4CF02F0E2
:10109000E9CF03F0000EE56E0F0EE56E420EE56E31
:1010A000400EE56E0350E56E0250E56E0150E56EB0
:1010B0000050E56EFFEC02F0006EF3CF01F0F4CFCC
:1010C00002F0E9CF03F0080EE12601C0F3FF005063
:1010D000E4CF03F0E4CF02F0E4CF01F0E4CF00F07E
:1010E000120000C0E5FF01C0E5FF02C0E5FF03C03C
:1010F000E5FFE0EC08F0006EF3CF01F0F4CF02F072
:10110000E9CF03F0000EE56E000EE56E030EE56E0E
:10111000E80EE56E0350E56E0250E56E0150E56E97
:101120000050E56EFFEC02F0006EF3CF01F0F4CF5B
:1011300002F0E9CF03F0080EE12601C0F3FF0050F2
:10114000E4CF03F0E4CF02F0E4CF01F0E4CF00F00D
:101150001200D9CFE5FFE1CFD9FF00C0E5FF01C004
:10116000E5FF02C0E5FF03C0E5FF04C0E5FF020E96
:10117000DBCF00F0030EDBCF01F0026A080E036E36
:10118000800E0014046ED8900036D89002360450B9
:10119000D8A402800150025C03E30150025E00808B
:1011A000032EEED70050E4CF04F0E4CF03F0E4CFF9
:1011B00002F0E4CF01F0E4CF00F0E4CFD9FF120059
:1011C00000C0E5FF01C0E5FF02C0E5FF03C0E5FF89
:1011D00004C0E5FF05C0E5FFB2CF00F0B3CF01F0DA
:1011E00088C002F089C003F0B2CF04F0B3CF05F09D
:1011F0000150055C02E10050045C04E288C002F08A
:1012000089C003F003C0E9FF02C0F4FF05C0F3FF8B
:101210000450E4CF05F0E4CF04F0E4CF03F0E4CFD2
:1012200002F0E4CF01F0E4CF00F0120000C0E5FFCF
:1012300001C0E5FF02C0E5FFFE0E0001806F010E58
:10124000816F8269000E016E800E006E800E026E4C
:10125000030EE56E0250E56E0150E56E0050E56E3E
:10126000000EE56E000EE56E000EE56EC60EE56E34
:101270008CEC03F0080EE126000EE56E0A0EE56E1A
:101280007EEC09F0020EE126E4CF02F0E4CF01F09B
:10129000E4CF00F01200D9CFE5FFE1CFD9FF00C0C5
:1012A000E5FF01C0E5FF02C0E5FF03C0E5FF020E58
:1012B000DBCF00F00044E844FC0B016E030E01108C
:1012C000C26EC2B2FED7C4CF00F0016A0050036EF6
:1012D000026AC3CF00F0016A0050022601500322C7
:1012E00003C0F3FF0250E4CF03F0E4CF02F0E4CFF9
:1012F00001F0E4CF00F0E4CFD9FF1200D9CFE5FF31
:10130000E1CFD9FF00C0E5FF01C0E5FF02C0E5FF66
:1013100003C0E5FF020EDBCF00F0030EDBCF01F0D0
:1013200000C002F001C003F0FF0E0026D8A00106A5
:101330000250031006E0FA0E026E0000022EFDD7E6
:10134000EFD7E4CF03F0E4CF02F0E4CF01F0E4CF35
:1013500000F0E4CFD9FF120000C0E5FF01C0E5FFB7
:1013600002C0E5FFFF0E006E1F0EC514016E026A7B
:10137000C7B4022A02500112015003E000060050D7
:10138000F3E100C001F00050D8B467EC0AF001505E
:10139000D880E866D890016A01360150E4CF02F0A7
:1013A000E4CF01F0E4CF00F01200D9CFE5FFE1CFA8
:1013B000D9FF00C0E5FF01C0E5FF020EDBCF00F062
:1013C000030EDBCF01F0A69EA69CA684F29E01C070
:1013D000A8FF00C0A9FF550EA76EAA0EA76EA68291
:1013E000A6B2FED7A694F28EE4CF01F0E4CF00F0CF
:1013F000E4CFD9FF1200D9CFE5FFE1CFD9FF00C07C
:10140000E5FF01C0E5FF020EDBCF00F0ACEC09F018
:10141000C586ACEC09F0C9CF01F0ACEC09F0005086
:1014200002E0C59A01D0C58AC5880150E4CF01F019
:10143000E4CF00F0E4CFD9FF1200D9CFE5FFE1CF30
:10144000D9FF00C0E5FF020EDBCF00F0A69CA69EF0
:1014500000C0A9FFA680A850E4CF00F0E4CFD9FFD8
:10146000120000C0E5FF01C0E5FF1F0EC514006EAD
:10147000016AC7B4012A015000120050F6E1E4CF1E
:1014800001F0E4CF00F01200D9CFE5FFE1CFD9FFA2
:1014900000C0E5FF020EDBCF00F0ACA2FED700C01B
:1014A000ADFFE4CF00F0E4CFD9FF1200E8AE04D0E6
:1014B000F3CFEAFFEE501200E8BC08D0E9CFF6FF08
:1014C000F3CFF7FFF86E0900F55012001200818A81
:1014D000C69A9496828682B803D082968286FBD77B
:1014E00094988298828894869488C68A1200200EE6
:1014F000AC6E900EAB6E0C0EAF6E000EE56E010E74
:10150000E56E7EEC09F0020EE12612003F0EC716D2
:10151000280EC66EC56A090EC86E948694889E967B
:10152000A19667EC0AF0819A1200620ED36E0F0E3C
:10153000936E816ACDEC0AF0F26AF28CA082F28E90
:10154000FFD71200D9CFE5FFE1CFD9FF020EDBCFE5
:10155000C9FFACEC09F0E4CFD9FF120012EEFFF0A6
:1015600022EEFFF0F86AA68EA69C3DEC06F095EC04
:101570000AF0FFD7E8AE05D0F3CFEAFFE4CFEEFFE5
:101580001200E8AC1200120000C0E5FF006A9EBA2B
:10159000002A0050E4CF00F01200810EB16EB36A51
:1015A000B26A0001886B896B1200010EC26E050ED3
:1015B000C16E940EC06E12000100081600008B0070
:1015C000000001000000B36AB26A0001886B896BF9
:1015D0001200ACEC09F0C584C5B4FED71200ACEC27
:1015E00009F0C582C5B2FED71200ACEC09F0C58087
:1015F000C5B0FED712000001882B01E3892B120031
:0A1600009EAAFED7AE5012000000B3
:00000001FF
